:10000000AD2800380319A828A8002008840021186A
:100010008317A001A101A81B15280008A000A81C97
:10002000A828840A0008A100A8281A200005031D9A
:10003000A00AA82800308A0028080739820701345E
:10004000023404340834103420344034803421081D
:1000500020040319A00A8030201AA1062019A10645
:10006000A018A106210DA00DA10DA828A301A20092
:10007000FF30A207031CA307031CA8280330A1001C
:10008000DF3044203828A101E83EA000A109FC305F
:10009000031C4D28A00703184A28A0076400A10FDD
:1000A0004A2820185328A01C572800005728080069
:1000B000A20002306628A20001306628A2000630A5
:1000C0006628A20004306628A2000530A800230894
:1000D0002102031D6D28220820020430031801307C
:1000E000031902302805031DFF30A828A501A4012B
:1000F0001030A600210DA40DA50D2208A40223088E
:10010000031C230FA50203188C282208A407230828
:100110000318230FA5070310A00DA10DA60B7A2825
:100120002008A8281030A800A101A001A70CA60C47
:10013000031CA0282208A00723080318230FA107E7
:10014000A10CA00CA50CA40CA80B96282408A82888
:10015000831303138312640008008316870185014B
:100160008312D801D9015808A0005908A100A301A1
:1001700000308A0164208A11031DC0288A119C2343
:10018000D80A0319D90A4408A0004508A1008A0129
:1001900027202008C4002108C5004408A000450805
:1001A000A1001230A200A3018A0176202408C60013
:1001B0002508C70001304607C80047080318013E5C
:1001C000C9004808A0004908A100A30101308A0124
:1001D00064208A11031DF0288A11AF258A119A2BF9
:1001E0004808A0004908A100A30102308A01642048
:1001F0008A11031DFF288A11D7258A119A2B4808D6
:10020000A0004908A100A30103308A0164208A11DB
:10021000031D0E298A1156268A119A2B4808A00020
:100220004908A100A30104308A0164208A11031D3A
:100230001D298A1173278A119A2B4808A0004908A2
:10024000A100A30105308A0164208A11031D402901
:100250000130D600D7015608A0005708A100A3011D
:100260000A308A015B208A11031D3E298A15582015
:10027000D60A0319D70A8A11031D2B298A119A2B32
:100280004808A0004908A100A30106308A016420A3
:100290008A11031D9A29831640088312A000831631
:1002A00041088312A1008A01272020088316C0007C
:1002B000831221088316C10040088312A000831610
:1002C00041088312A1001030A200A3018A01762008
:1002D00024088316C200831225088316C300043045
:1002E0004207C40043080318013EC5000130C600A0
:1002F000C7018312831646088312A000831647089D
:100300008312A100831645088312A30083164408B4
:1003100083128A015B208A11031D98298A15C22045
:100320008316C60A0319C70A8A118312031D7A2984
:100330008A119A2B4808A0004908A100A3010730A0
:100340008A0164208A11031DF42983164008831250
:10035000A000831641088312A1008A0127202008EB
:100360008316C000831221088316C100400883123F
:10037000A000831641088312A1001030A200A3013F
:100380008A01762024088316C2008312250883166A
:10039000C30004304207C40043080318013EC500EF
:1003A0000130C600C7018312831646088312A000DD
:1003B000831647088312A100831645088312A30001
:1003C0008316440883128A015B208A11031DF229D7
:1003D0008A15E8208316C60A0319C70A8A118312F0
:1003E000031DD4298A119A2B4808A0004908A100AE
:1003F000A30108308A0164208A11031D032A8A158B
:100400000E218A119A2B4808A0004908A100A301D7
:1004100009308A0164208A11031D2E2A83160130B7
:10042000C800C9018312831648088312A0008316EE
:1004300049088312A100A3010A308A015B208A11B6
:10044000031D2C2A8A1593218316C80A0319C90A89
:100450008A118312031D132A8A119A2B4808A000BF
:100460004908A100A3010A308A0164208A11031DF2
:100470003D2A8A15DE218A119A2B4808A0004908D6
:10048000A100A3010B308A0164208A11031D4C2AAC
:100490008A157F228A119A2B4808A0004908A100DA
:1004A000A3010C308A0164208A11031D772A831668
:1004B0000130C800C9018312831648088312A000C6
:1004C000831649088312A100A3010A308A015B2028
:1004D0008A11031D752A8A1505238316C80A031974
:1004E000C90A8A118312031D5C2A8A119A2B4808B3
:1004F000A0004908A100A3010D308A0164208A11DF
:10050000031DB92A3808A0003908A1008A01272054
:100510002008B8002108B9003808A0003908A10057
:100520000630A200A3018A0176202408BA0025081B
:10053000BB0001303A07BC003B080318013EBD0078
:100540000130D000D1015008A0005108A1003D08A1
:10055000A3003C088A015B208A11031DB72A8A1573
:100560004B23D00A0319D10A8A11031DA32A8A1129
:100570009A2B4808A0004908A100A3010E308A0167
:1005800064208A11031DC82A8A1594238A119A2B84
:100590004808A0004908A100A3010F308A01642087
:1005A0008A11031D2F2B8C30E400E5016408A000A4
:1005B0006508A100A30164308A0161208A11031D2E
:1005C000F12A8A151D240A30E40200308A1103182A
:1005D000ED2A013E8A110318F12AE5028A11031857
:1005E000D62A6430E400E5016408A0006508A10093
:1005F000A30150308A0161208A11031D0F2B8A1537
:100600001D240530E40200308A1103180B2B013E33
:100610008A1103180F2BE5028A110318F42A831696
:100620000130CA00CB01831283164A088312A0004E
:1006300083164B088312A100A30107308A015B20B7
:100640008A11031D2D2B8A151D248316CA0A03192E
:10065000CB0A8A118312031D142B8A119A2B480886
:10066000A0004908A100A30110308A0164208A116A
:10067000031D5A2B6E30F200F3017208A0007308BC
:10068000A100A30150308A0161208A11031D582B5B
:100690008A1566240A30F20200308A110318542B9E
:1006A000013E8A110318582BF3028A1103183D2BBF
:1006B0008A119A2B4808A0004908A100A301113013
:1006C0008A0164208A11031D7D2B0130D200D301E1
:1006D0005208A0005308A100A30105308A015B2045
:1006E0008A11031D7B2B8A15EC24D20A0319D30A25
:1006F0008A11031D682B8A119A2B4808A00049080B
:10070000A100A30113308A0158208A11031D932BE5
:100710004808A0004908A100A30112308A01642002
:100720008A11031D9A2B8A1525250330A300E83072
:100730008A0137208A01B32883161930B200B30129
:100740008312831632088312A000831633088312A3
:10075000A1000B30A300B8308A015B208A11031D71
:10076000F22B0130BE00BF013E08A0003F08A100EF
:10077000A30102308A015B208A11031DE52B3F3063
:10078000870007308500831633088312A100831683
:10079000320883128A0144208701850183163208BA
:1007A000883CDC003308031C013E133CDD005D087F
:1007B0008312A10083165C0883128A014420BE0ABA
:1007C0000319BF0A8A11031DB42B19308316B2070F
:1007D0008A118312031CA12B8316B30A8A11831278
:1007E000031DA12B8316B830B2000B30B300831267
:1007F000831632088312A000831633088312A100E7
:100800001130A30094308A015B208A11031D492C0A
:100810000130BE00BF013E08A0003F08A100A301B7
:1008200002308A015B208A11031D3C2C3F30870077
:1008300007308500831633088312A100831632081F
:1008400083128A0144208701850183163208883C7F
:10085000DC003308031C013E133CDD005D088312FD
:10086000A10083165C0883128A014420BE0A031982
:10087000BF0A8A11031D0B2C0A308316B2078A1196
:100880008312031CF82B8316B30A8A118312031DEB
:10089000F82B83169430B2001130B3008312831604
:1008A00032088312A000831633088312A10013308C
:1008B000A30088308A015B208A11031DA02C01301F
:1008C000BE00BF013E08A0003F08A100A301023006
:1008D0008A015B208A11031D932C3F30870007306B
:1008E0008500831633088312A10083163208831211
:1008F0008A0144208701850183163208883CDC0088
:100900003308031C013E133CDD005D088312A10087
:1009100083165C0883128A014420BE0A0319BF0AA9
:100920008A11031D622C05308316B2078A118312C7
:10093000031C4F2C8316B30A8A118312031D4F2CFC
:10094000080083168830CC001330CD008312831644
:100950004C088312A00083164D088312A1001130A9
:10096000A30094308A0161208A11031DFB2C013001
:10097000C200C3014208A0004308A100A301023045
:100980008A015B208A11031DEB2C3F308700073062
:10099000850083164D088312A10083164C0883122C
:1009A0008A01442087018501883083164C07DE00C8
:1009B00013300318013E4D07DF005F088312A100CA
:1009C00083165E0883128A014420C20A0319C30AEF
:1009D0008A11031DBA2C23308316CC0200308A11F1
:1009E00083120318F72C013E8A110318FB2CCD0249
:1009F0008A110318A72C83169430CC001130CD0037
:100A0000831283164C088312A00083164D088312AC
:100A1000A1000730A300D0308A0161208A11031D94
:100A2000552D0130C200C3014208A0004308A100B7
:100A3000A30102308A015B208A11031D452D3F303E
:100A400087000730850083164D088312A1008316A6
:100A50004C0883128A01442087018501883083165F
:100A60004C07DE0013300318013E4D07DF005F081E
:100A70008312A10083165E0883128A014420C20AF1
:100A80000319C30A8A11031D142D14308316CC02D6
:100A900000308A1183120318512D013E8A11031868
:100AA000552DCD028A110318012D8316D030CC00AC
:100AB0000730CD00831283164C088312A0008316E2
:100AC0004D088312A100A30100308A0161208A1120
:100AD000031DAE2D0130C200C3014208A00043082F
:100AE000A100A30102308A015B208A11031D9E2D03
:100AF0003F3087000730850083164D088312A10020
:100B000083164C0883128A014420870185018830AE
:100B100083164C07DE0013300318013E4D07DF003B
:100B20005F088312A10083165E0883128A014420A5
:100B3000C20A0319C30A8A11031D6D2D0A308316D8
:100B4000CC0200308A1183120318AA2D013E8A11AB
:100B50000318AE2DCD028A1103185B2D0800013059
:100B6000EE00EF016E08A0006F08A100A3010A309B
:100B70008A015B208A11031DD62D3230DA00DB0199
:100B80003F308700073085005B08A3005A088A01C0
:100B90003720870185015B08A3005A088A013720A6
:100BA000EE0A0319EF0A8A11031DB22D0800643002
:100BB000E800E9016808A0006908A100A301463027
:100BC0008A0161208A11031DF52D8A1132260A300F
:100BD000E80200308A110318F12D013E8A11031832
:100BE000F52DE9028A110318DA2D4630E800E901F3
:100BF0006808A0006908A100A30132308A016120C1
:100C00008A11031D132E8A1132260530E8020030A6
:100C10008A1103180F2E013E8A110318132EE902C0
:100C20008A110318F82D83160130A800A901831238
:100C3000831628088312A000831629088312A100B6
:100C4000A30107308A015B208A11031D312E8A110E
:100C500032268316A80A0319A90A8A118312031DD2
:100C6000182E080012308700023085006908A300A2
:100C700068088A0137201130870004308500690830
:100C8000A30068088A013720383087008501690889
:100C9000A30068088A0137201430870001308500DE
:100CA0006908A30068088A01372008009630F00020
:100CB000F1017008A0007108A100A30164308A014D
:100CC00061208A11031D742E8A11B1260F30F002A3
:100CD00000308A110318702E013E8A110318742EF9
:100CE000F1028A110318592E6430F000F1017008E6
:100CF000A0007108A100A3011E308A0161208A11A1
:100D0000031D922E8A11B1260A30F00200308A119A
:100D100003188E2E013E8A110318922EF1028A11B9
:100D20000318772E83160130AA00AB0183128316B5
:100D30002A088312A00083162B088312A100A301A6
:100D400007308A015B208A11031DB02E8A11B1265B
:100D50008316AA0A0319AB0A8A118312031D972E60
:100D6000080024308700043085007108A300700853
:100D70008A01372010308700023085007108A300F7
:100D800070088A0137208701013085007108A300AF
:100D900070088A013720093087000130850071080A
:100DA000A30070088A0137201030870002308500C8
:100DB0007108A30070088A0137208701043085007C
:100DC0007108A30070088A01372087010730850069
:100DD0007108A30070088A01372018308700850148
:100DE0007108A30070088A0137200130870085014F
:100DF0007108A30070088A01372007308700850139
:100E00007108A30070088A01372018308700850117
:100E10007108A30070088A0137208701013085001E
:100E20007108A30070088A0137200930870001305B
:100E300085007108A30070088A01372012308700EE
:100E400085017108A30070088A01372004308700EB
:100E50007108A30070088A0137202430870004300D
:100E600085007108A30070088A01372012308700BE
:100E700085017108A30070088A01372001308700BE
:100E80007108A30070088A013720073087008501A8
:100E90007108A30070088A0137203030870071087C
:100EA000A30070088A01372087010430850071088B
:100EB000A30070088A013720073085007108A3005D
:100EC00070088A0137203030870085017108A3003F
:100ED00070088A013720643087007108A300700809
:100EE0008A01372008008316C830A200A3018312AC
:100EF000831622088312A000831623088312A10000
:100F0000A30164308A0161208A11031D992F8A117F
:100F1000B02714308316A20200308A1183120318FE
:100F2000952F013E8A110318992FA3028A110318E5
:100F3000782F0130CC00CD014C08A0004D08A10055
:100F4000A30107308A015B208A11031DAF2F8A118C
:100F5000B027CC0A0319CD0A8A11031D9C2F080063
:100F60005030F600F7010130870085017708A300B3
:100F700076088A0137200A3087007708A3007608B0
:100F80008A01372014308700013085007708A300DC
:100F900076088A01372020308700023085007708E4
:100FA000A30076088A01372087010430850077087E
:100FB000A30076088A01372004308700850177086E
:100FC000A30076088A013720223087007708A30023
:100FD00076088A01372011308700043085007708B1
:100FE000A30076088A013720083087000230850088
:100FF0007708A30076088A01372087010130850031
:101000007708A30076088A0137208701043085001D
:101010007708A30076088A01372020308700023045
:1010200085007708A30076088A01372014308700EE
:10103000013085007708A30076088A0137200A303E
:10104000870085017708A30076088A0137200130E0
:1010500087007708A30076088A01372087010130CE
:1010600085007708A30076088A01372008308700BA
:10107000023085007708A30076088A0137201130F6
:101080008700043085007708A30076088A0137209E
:101090002230870085017708A30076088A0137206F
:1010A000043087007708A30076088A0137200800FB
:1010B0005030F800F9014008A0004108A100A30148
:1010C00000308A0164208A15031D6A2809308700D0
:1010D000013085004008A0004108A100A3010030B4
:1010E0008A015E208A15031D79280F3087000130A0
:1010F0008500C00A0319C10A7908A30078088A018B
:10110000372012308700023085007908A300780864
:101110008A01372027308700043085007908A30032
:1011200078088A0137203830870085017908A300C4
:1011300078088A0137202430870007308500790835
:10114000A30078088A01372012308700023085001A
:101150007908A30078088A01372009308700073012
:1011600085007908A30078088A0137203830870085
:1011700085017908A30078088A01372007308700A5
:10118000850108006430FA00FB0103308700063057
:1011900085007B08A3007A088A0137203830870051
:1011A00085017B08A3007A088A0137200630870072
:1011B000033085007B08A3007A088A013720383085
:1011C000870085017B08A3007A088A013720080080
:1011D0006430EA00EB0102308700053085006B08BF
:1011E000A3006A088A0137203830870085016B0820
:1011F000A3006A088A013720053087000230850085
:101200006B08A3006A088A013720383087008501FF
:101210006B08A3006A088A01372008002030FC0010
:101220000330FD005E30FE000130FF0087018501C4
:101230007D08A3007C088A013720063087008501DD
:101240007D08A3007C088A013720343087007D08A0
:10125000A3007C088A0137202030870006308500F3
:101260007D08A3007C088A013720223087000630E1
:1012700085007D08A3007C088A013720363087006E
:10128000063085007D08A3007C088A0137203730AE
:101290008700063085007D08A3007C088A0137207E
:1012A0003F308700063085007D08A3007C088A0156
:1012B00037203F308700073085007D08A3007C0879
:1012C0008A013720870185017F08A3007E088A01F3
:1012D00037203F308700073085007F08A3007E0855
:1012E0008A013720870185017F08A3007E088A01D3
:1012F00037203F308700073085007F08A3007E0835
:101300008A013720870185017F08A3007E088A01B2
:1013100037203F308700073085007F08A3007E0814
:101320008A01372008003C30F400F501850187016F
:101330007508A30074088A013720043087007508F7
:10134000A30074088A013720023087007508A300C3
:1013500074088A013720013087007508A3007408DB
:101360008A013720203087007508A30074088A019D
:101370003720103087007508A30074088A013720D1
:10138000083087007508A30074088A0137200430EC
:10139000850087017508A30074088A013720023090
:1013A00085007508A30074088A0137200130850084
:1013B0007508A30074088A0137200800CA01CB0110
:1013C0004A08A0004B08A100A30110308A015B204D
:1013D0008A15031D7E2A4B088A15031D412A4A08D7
:1013E000A200103C8A15031C412A0310220DA207FB
:1013F0008A150A22A000A20A8A150A22A100A20ABE
:101400008A150A228A0101202008EC002108ED003B
:101410008A15412A0A308A0022088207FA340034E9
:101420000034E13400340034C834003400349634DD
:10143000003400346434003400345A34003400344E
:101440005034003400344634003400344134003425
:1014500000343E34003400343C34003400343A3438
:10146000003400343834003400343534003400346F
:101470003234003400343234003400343234003436
:101480000034850187016D08A3006C088A013720AC
:10149000103087006D08A3006C088A0137202A30BD
:1014A0008700023085006D08A3006C088A01372090
:1014B000850187016D08A3006C088A01372005307B
:1014C0008700053085006D08A3006C088A0137206D
:1014D000850187016D08A3006C088A0137202A3036
:1014E0008700023085006D08A3006C088A01372050
:1014F000CA0A0319CB0A8A15031DE02908008230A5
:10150000DC00DD015C08A0005D08A100A3016430DF
:101510008A0161208A15031D9D2A8A15DA220A3064
:10152000DC0200308A150318992A013E8A15031837
:101530009D2ADD028A150318822A6430DC00DD0151
:101540005C08A0005D08A100A3014B308A01612066
:101550008A15031DBB2A8A15DA220530DC02003009
:101560008A150318B72A013E8A150318BB2ADD0223
:101570008A150318A02A83160130AE00AF0183122A
:1015800083162E088312A00083162F088312A10051
:10159000A3010A308A015B208A15031DD92A8A1506
:1015A000DA228316AE0A0319AF0A8A158312031DC5
:1015B000C02A08002030870085015D08A3005C0870
:1015C0008A01372014308700043085005D08A300AD
:1015D0005C088A0137200A308700023085005D08E8
:1015E000A3005C088A0137200130870001308500A4
:1015F0005D08A3005C088A013720870185015D082A
:10160000A3005C088A01372008005030DE00DF01AB
:101610008701043085005F08A3005E088A01372037
:10162000023085005F08A3005E088A013720083079
:10163000870085015F08A3005E088A0137202030FB
:1016400087005F08A3005E088A01372010308700FA
:101650005F08A3005E088A013720013087005F0819
:10166000A3005E088A013720043087005F08A300CA
:101670005E088A013720023087005F08A3005E08F9
:101680008A0137200130850087015F08A3005E08CA
:101690008A01372008005030E000E1010130870066
:1016A00085016108A30060088A01372002308700A5
:1016B00085016108A30060088A0137200430870093
:1016C00085016108A30060088A0137202030870067
:1016D0006108A30060088A01372087010430850073
:1016E0006108A30060088A0137200830870085015F
:1016F0006108A30060088A01372010308700610864
:10170000A30060088A013720870102308500610844
:10171000A30060088A013720013085006108A3001A
:1017200060088A01372008001E30E200E3016208E9
:10173000A0006308A100A30132308A015B208A1552
:10174000031DD82B0230850087016308A3006208BF
:101750008A0137201030870085016308A3006208E2
:101760008A013720023087006308A30062088A01DB
:101770003720053087006308A30062088A013720FC
:10178000283087006308A30062088A013720870198
:10179000053085006308A30062088A013720053000
:1017A000E2078A15031C972BE30A8A15031D972B62
:1017B0003230E200E3016208A0006308A100A30147
:1017C00064308A015B208A15031D1C2C02308500C1
:1017D00087016308A30062088A0137201030870060
:1017E00085016308A30062088A0137200230870060
:1017F0006308A30062088A01372005308700630868
:10180000A30062088A013720283087006308A300FC
:1018100062088A0137208701053085006308A3002C
:1018200062088A0137200A30E2078A15031CDB2B85
:10183000E30A8A15031DDB2B0800273087000730D9
:1018400085006508A30064088A0137202F308700CF
:10185000063085006508A30064088A0137202F3010
:101860008700053085006508A30064088A013720D9
:101870002F308700033085006508A30064088A01C3
:1018800037200F308700073085006508A300640803
:101890008A0137202B308700073085006508A300B8
:1018A00064088A0137202D308700073085006508DD
:1018B000A30064088A0137202E3087000730850096
:1018C0006508A30064088A013720080004308700F7
:1018D00085017308A30072088A013720243087002D
:1018E0007308A30072088A0137200430850073084A
:1018F000A30072088A013720063085007308A30010
:1019000072088A013720203087000730850073086D
:10191000A30072088A013720083087007308A300EB
:1019200072088A0137200930870003308500730868
:10193000A30072088A0137200B3087000130850030
:101940007308A30072088A0137201B3087008501C5
:101950007308A30072088A01372013308700023011
:1019600085007308A30072088A01372012308700AF
:10197000063085007308A30072088A0137203030D2
:101980008700063085007308A30072088A0137209B
:1019900024308700063085007308A30072088A018E
:1019A0003720043085007308A30072088A013720AD
:1019B00085017308A30072088A013720043087006C
:1019C0007308A30072088A01372087017308A300F7
:1019D00072088A013720080017308700023085001E
:1019E00064308A013620363087000130850064304B
:1019F0008A0136203C3087000430850064308A013B
:101A00003620313087000630850064308A01362068
:101A1000123087000730850064308A0136201C3080
:101A200087000330850064308A0136203930870012
:101A30000130850064308A0136201B308700043075
:101A4000850064308A01362008002830E600E7016E
:101A5000831636088312A000831637088312A1006C
:101A60008A01272020088316B600831221088316D6
:101A7000B70036088312A000831637088312A1002E
:101A80001E30A200A3018A01762024088316B80024
:101A9000831225088316B9000A303807BA003908BE
:101AA0000318013EBB000130B400B5018312831658
:101AB00034088312A000831635088312A100831610
:101AC0003B088312A30083163A0883128A015B2025
:101AD0008A15031DAC2E831624088312A0008316DA
:101AE00025088312A1008A01272020088316A4005C
:101AF000831221088316A50024088312A0008316F0
:101B000025088312A1000230A200A3018A017620D9
:101B100024088316BC00831225088316BD003C08E8
:101B20008312A00083163D088312A100A301003098
:101B30008A0164208A15031D9F2D8A152B2E83167A
:101B40003C088312A00083163D088312A100A30164
:101B500001308A0161208A15031D2B2E8316D001C6
:101B6000D1014E088312A00083164F088312A100F2
:101B70008A01272020088316CE00831221088316AD
:101B8000CF004E088312A00083164F088312A100D5
:101B90000630A200A3018A01762024088316D00013
:101BA000831225088316D10050088312A0008316E3
:101BB00051088312A100A30100308A0164208A1514
:101BC000031DE92D83160130D400D50183128A1537
:101BD0001F2E83160130D400D5010130D200D3016D
:101BE0008312831652088312A000831653088312AF
:101BF000A100831651088312A30083165008831294
:101C00008A015B208A15031D1F2E83165408831238
:101C1000A600831655088312A7000230A200A30174
:101C20008A0192208316D400831225088316D500DA
:101C3000D20A0319D30A8A158312031DF12D8316C4
:101C400054088312870085016708A30066088A018B
:101C500037208A15A42E831656088312A0008316F7
:101C600057088312A1008A01272020088316D60076
:101C7000831221088316D70056088312A00083160A
:101C800057088312A1000330A200A3018A01762025
:101C900024088316D800831225088316D900580813
:101CA0008312A000831659088312A100A3010030FB
:101CB0008A0164208A15031D642E83160130DA0020
:101CC000DB0183128A159A2E83160130DA00DB01BC
:101CD0000130B000B1018312831630088312A000D6
:101CE000831631088312A100831659088312A300BA
:101CF0008316580883128A015B208A15031D9A2EC9
:101D000083165A088312A60083165B088312A70065
:101D10000230A200A3018A0192208316DA00831206
:101D200025088316DB00B00A0319B10A8A1583124D
:101D3000031D6C2E83165A088312850087016708DD
:101D4000A30066088A0137208316B40A0319B50A6E
:0A1D50008A158312031D572D0800A9
:02400E00FC3F75
:00000001FF
